:200000000200E3758920758BFD758D020078E4F50AF50B050BE50B7002050AB410F5E50A58
:20002000B427F0E4F50AF50B050BE50B7002050AB410F5E50AB427F0E4F50AF50B050BE546
:200040000B7002050AB410F5E50AB427F0E4F50AF50B050BE50B7002050AB410F5E50AB4E1
:2000600027F0E4F50AF50B050BE50B7002050AB410F5E50AB427F022C0E0C0D0D3E50994EB
:2000800080E508940C5024C28CB290750A00750B00050BE50B7002050A641E450A70F2B2EA
:2000A000900509E50970110508800DC28C750800750901B29112000E758CFE758A0CD28C84
:2000C000D0D0D0E032750800750901758901C290C29112000E758CFE758A0CD2AFD2A9D206
:1000E0008C80FE787FE4F6D8FD75810B0200C5F5A3
:00000001FF
